:1000000027C036C035C034C033C032C031C030C064
:100010002FC02EC02DC0C0C02BC02AC029C028C0F0
:1000200027C000003A00370000003B003800010103
:100030000101010101010202020102040810204035
:10004000800402010000000000040302010000001F
:1000500011241FBECFE5D1E0DEBFCDBF20E0A0E67A
:10006000B0E001C01D92A936B207E1F7DFD020C190
:10007000C7CFECE4F0E02491E1E4F0E09491E6E312
:10008000F0E0E491EE23C1F0222329F0223021F1A7
:10009000A0F42130E9F0F0E0EE0FFF1FE85DFF4F24
:1000A000A591B4912FB7F894811119C08C91E92FC3
:1000B000E095E823EC932FBF0895233029F02430F6
:1000C00051F72FB52F7D02C02FB52F772FBDE3CF6E
:1000D00020B72F7720BFDFCF20B72F7DFBCFEC914C
:1000E000E92BE8CF3FB7F8948091650090916600C6
:1000F000A0916700B091680022B708B600FE05C065
:100100002F3F19F00196A11DB11D3FBFBA2FA92F96
:10011000982F8827BC01CD01620F711D811D911D93
:1001200046E0660F771F881F991F4A95D1F70895FB
:100130008F929F92AF92BF92CF92DF92EF92FF92F7
:10014000D1DF4B015C0188EEC82E83E0D82EE12C74
:10015000F12CC8DF681979098A099B09683E734048
:1001600081059105B0F321E0C21AD108E108F10838
:1001700088EE880E83E0981EA11CB11CC114D10426
:10018000E104F10431F7FF90EF90DF90CF90BF9042
:10019000AF909F908F9008951F920F920FB60F927D
:1001A00011242F933F938F939F93AF93BF9380918D
:1001B000610090916200A0916300B0916400309161
:1001C000600020E3230F2D3758F54096A11DB11D87
:1001D000209360008093610090936200A09363007D
:1001E000B09364008091650090916600A0916700D3
:1001F000B09168000196A11DB11D80936500909398
:100200006600A0936700B0936800BF91AF919F9183
:100210008F913F912F910F900FBE0F901F901895C7
:1002200023EB230F4196A11DB11DD2CF789480B747
:10023000826080BF80B7816080BF83B7826083BFE8
:1002400083B7816083BF89B7816089BF1EBC8EB5CB
:1002500082608EBD8FB581608FBD3298319A309AA1
:10026000379AE1E4F0E02491E6E3F0E0849188231A
:1002700099F090E0880F991FFC01EE5DFF4FA5916A
:10028000B491FC01E85DFF4F859194918FB7F8948C
:10029000EC91E22BEC938FBFC0E0D0E081E0E9DE8F
:1002A00047DF80E0E6DE44DF2097C1F3A9DEF6CF2A
:0402B000F894FFCFF0
:00000001FF
